:020000040000FA
:1000000000308A002D28000022308400831300086D
:10001000031918280130F800F701F70B0D28F80B29
:100020000C284A30F700F70B13281628800B0A28F3
:1000300000341230A302031C2C28233084008313C5
:10004000FC3080050310800C800C000803192C285C
:100050002A280000800B29280034840183131F30D4
:100060008305623083168F000F081F129F121B0832
:1000700080399B0007309C0081131F129F121B08C0
:1000800080399B0083121F10940183160108C73921
:1000900008388100831290010030F800920000308F
:1000A0008316920007309C00050885000330F70096
:1000B000F70B58281C0883120D1383169D01061593
:1000C0008312061DB1288316861083128614013010
:1000D000A20004200230A200F730A3001920A20BD6
:1000E0006C2883168610831286108316851183125E
:1000F00085150130A20004200230A200F730A300D1
:100100001920A20B7E288316851183128511831670
:100110000511831205150130A20004200230A2004F
:10012000F730A3001920A20B902883160511831223
:10013000051183160510831205140130A200042056
:100140000230A200F730A3001920A20BA2288316C8
:100150000510831205100A30A200042083165F28C0
:10016000831283160615831206192329A10121087B
:10017000633C031CEC28831686108312861401301E
:10018000A200042083168610831286108316851120
:10019000831285150130A200042083168511831275
:1001A000851183160511831205150130A200042064
:1001B0008316051183120511831605108312051489
:1001C0000130A200042083160510831205100A30A6
:1001D000A2000420A10AB728A1012108633C031C46
:1001E000222983168610831286140230A20004206E
:1001F0008316861083128610831685118312851547
:100200000230A20004208316851183128511831603
:100210000511831205150230A20004208316051172
:100220008312051183160510831205140230A200F3
:10023000042083160510831205100A30A200042042
:0C024000A10AED28B12883165F28630096
:04400E00783FFF3FB9
:00000001FF
